:100000000C943A000C9457000C9457000C94570031
:100010000C9457000C9459000C9457000C94570002
:100020000C9457000C94A9000C9457000C94710088
:100030000C9457000C9457000C9446010C944B01FF
:100040000C9457000C9457000C9457000C945700D4
:100050000C9457000C946F010C9457000C945700AB
:100060000C9457000C9457003F065B4F666D7D075C
:100070007F6F394011241FBECFEFD8E0DEBFCDBF68
:1000800011E0A0E0B1E0E4EAF9E002C005900D92D1
:10009000A630B107D9F721E0A6E0B1E001C01D927A
:1000A000A531B207E1F70E94BC030C94D0040C9474
:1000B00000008F938FB78F93EF93FF9389B1809553
:1000C0008C7F8093080185E080930901EFE6F0E0E2
:1000D000808182608083FF91EF918F918FBF8F919C
:1000E00018951F921FB61F9211248F939F93809192
:1000F0000901882389F080910901815080930901C9
:1001000089B180958C7F90910801981759F095E0FE
:1001100090930901809308019F918F911F901FBEBA
:100120001F901895809109018111F6CF81E080938D
:100130000B018091080180930A0180910A0180954A
:1001400080788093110180916F008D7F80936F0084
:10015000E3CF1F920F920FB60F9211242F933F936C
:100160004F935F936F937F938F939F93AF93BF93BF
:10017000EF93FF93809114018F5F8093140180911E
:1001800014018C3309F049C01092140180911301BD
:100190008F5F80931301809113018C3359F5109276
:1001A0001301809112018F5F8093120180911201DF
:1001B000883101F51092120180910D018F5F8093BB
:1001C0000D0160910D01673059F410920D0180917D
:1001D0000C01209114010E949A04920F9093140133
:1001E00080910C012091140167E00E949A04820F13
:1001F000809314019091120180910E01981336C0E2
:100200009091130180910F01981330C081E0809389
:1002100010018EE887BD87E488BD80911001882396
:1002200051F080911101882321F08091140180FD0B
:1002300026C00E94B303809164008E7F8093640087
:1002400080917A00806480937A00FF91EF91BF9152
:10025000AF919F918F917F916F915F914F913F915E
:100260002F910F900FBE0F901F9018958091100145
:10027000882399F2109210010E94B303CECF80918F
:100280006E00866080936E00429AD5CF8F9386E091
:1002900086B98F9118951F920F920FB60F92112465
:1002A0002F933F934F935F936F937F938F939F937E
:1002B000AF93BF93EF93FF930E944601FF91EF919D
:1002C000BF91AF919F918F917F916F915F914F916E
:1002D0003F912F910F900FBE0F901F9018951F9276
:1002E0001FB61F9211248F939F9380910201882340
:1002F00011F18091790090910101805A8095890FC8
:100300009927991F95958795809301018091070101
:10031000811106C080E680937C00109202012D9A24
:10032000809164008160809364009F918F911F9001
:100330001FBE1F90189580917900829586958770D1
:10034000909100018E5F883008F087E0890F8093DC
:1003500000018091000190E09595879580930001C0
:100360008EE680937C0081E0809302012D98D8CFA7
:10037000109207010895439A81E080930701E8E60F
:10038000F0E08081846080836091060181E00E94BA
:100390004603089582E0809307014398E8E6F0E081
:1003A00080818B7F80830895259A87B18E6087B97D
:1003B0008BB18C6F8BB980916D008C6F80936D00C9
:1003C00080916800846080936800439A80917E00E9
:1003D000816080937E0080917A008C6880937A009F
:1003E0008EE680937C008091B60080628093B60098
:1003F0001092B20085E08093B1008091B6008571C3
:10040000E1F7109280008CE08093810080E290E020
:10041000909389008093880082E084BD85BD8EE83A
:1004200087BD80917000816080937000809164002E
:10043000876880936400789408950F931F93CF93F7
:10044000DF9330911201809112012AE0622F0E9405
:100450008E04092FCAE03A3020F0832F0E948E04C8
:10046000C82F10911301D0911301809106010E94B1
:100470004F038091140181700E9499036C2F80E0DA
:100480000E947103602F81E00E947103CAE0812FF6
:100490006C2F0E948E04682F82E00E9471038D2FC2
:1004A0006C2F0E948E04692F83E00E947103DF91FC
:1004B000CF911F910F9108950F931F93CF93DF93C7
:1004C00030910E0180910E012AE0622F0E948E046D
:1004D000092FCAE03A3020F0832F0E948E04C82FE3
:1004E00010910F01D0910F01809106010E944F03DE
:1004F0008091140181700E9499036C2F80E00E940A
:100500007103602F81E00E947103CAE0812F6C2F7C
:100510000E948E04682F82E00E9471038D2F6C2F41
:100520000E948E04692F83E00E947103DF91CF91B6
:100530001F910F9108951F93CF93DF9380910C012A
:10054000C0910C01C7FD81956AE00E948E04182FAE
:10055000D92F809106010E944F0380E00E949903E9
:100560006AE080E00E9485036BE0C7FF6CE081E0F9
:100570000E948503612F82E00E9471036D2F83E04A
:100580000E947103DF91CF911F9108959091100106
:10059000992321F09091140190FD06C0803429F038
:1005A000803631F00E941D0208950E945C02089579
:1005B0000E949B020895000000000000000000005F
:1005C00008950F931F93CF93DF93C82FD8E04598DA
:1005D0000E94DB020C2F10E0C0FF25C0449A459A10
:1005E0000E94DB0215950795C02FD15081F74598E1
:1005F0003C98449A0E94DB0286B1C82FC07184FFE8
:1006000003C03C9A4498C1E00E94DB02459A0E94D4
:10061000DB0245980E94DB023C9A8C2FDF91CF9140
:100620001F910F9108954498DACF87B1806387B9FD
:1006300008950E941503449A459A0E94DB0244984B
:10064000089587B18F7C87B9089545980E94DB0291
:1006500044980E94DB02459A0E94DB02449A0E9461
:1006600021030895CF93C0E08111C8E0683008F0FD
:1006700067E0C62BC09304010E9419038C2F806889
:100680000E94E1020E942503CF9108950E94320347
:1006900008956091040167700E9432030895682FE5
:1006A00067708091040188700E9432030895CF938F
:1006B000DF93C82FD62F0E94190384E40E94E10221
:1006C0000E9425030E9419038C2F8370806C0E9466
:1006D000E1028D2F0E94E1020E942503DF91CF915C
:1006E00008956A3080F4E62FF0E0E859FF4F6491F6
:1006F000813031F4909103019078692B609303016C
:100700000E945703089560E0F3CF6C3080F4E62F29
:10071000F0E0E859FF4F6491813031F4909103018A
:100720009078692B609303010E945703089560E05D
:10073000F3CF90910301882349F0906890930301CF
:100740006091030181E00E94570308959F77F6CFDF
:10075000CF93C0E060E08C2F0E945703CF5FC4307E
:10076000C9F7CF910895EEE6F0E08081897F80831C
:1007700088B1897F88B908950E94D40167E081E03B
:100780000E94460381E00E944903E9B0DE2DD09526
:10079000DC7FC0E085E0D82E98E1E92EF12C0CE357
:1007A00010E022E0C22ED092B10080910B0188238C
:1007B000E9F110920B0180910A018D27D0910A0175
:1007C000CD2FC077C03409F44BC058F4C031D1F0FC
:1007D000C03241F19D2F9C709C3009F470C0C0E084
:1007E00025C0C036B9F78D2382FD5EC083FF1EC0D1
:1007F00080910C018E39D4F080910C01815080934E
:100800000C0114C0282F2D2322FD3AC023FF0EC057
:100810008091120190E00196B7010E94A804809394
:10082000120104C0109210010E94B30380910701CD
:10083000813009F44CC0823009F466C081116BC06C
:10084000809100018093060180910101873520F499
:10085000C09206010E94BB018C2F0E94C6023DC0BF
:10086000282F2D2322FD16C023FFE0CF80910E01FB
:1008700090E00196B7010E94A80480930E01D6CFA4
:100880008091130190E00196B8010E94A804809322
:100890001301BCCF80910F0190E00196B8010E9436
:1008A000A80480930F01E0CF90910C0193360CF0D7
:1008B0009DCF90910C019F5F90930C0197CF8D235A
:1008C000C82FCC7009F4B2CF1092140188CF809158
:1008D0000101833588F40E94CA018091B6008571B8
:1008E000E1F783B7817F83BF83B7816083BF88953A
:1008F00083B78E7F83BF57CF80910101883508F47D
:10090000ABCF10920701A8CF80910101843528F365
:100910000E94BB01E2CF10920701DFCF991B79E063
:1009200004C0991F961708F0961B881F7A95C9F77F
:100930008095089587FB082E062687FD819567FD23
:1009400061950E948E040EF4919507FC819508959F
:1009500097FB072E16F4009407D077FD09D00E946C
:10096000BC0407FC05D03EF4909581959F4F0895F7
:10097000709561957F4F0895AA1BBB1B51E107C07D
:10098000AA1FBB1FA617B70710F0A61BB70B881F1F
:10099000991F5A95A9F780959095BC01CD010895AE
:0409A000F894FFCFF9
:0609A400075C01FF0F00DB
:00000001FF
